:100000006F2B8207FF34FF34FF34FF34FF34FF349B
:10001000FF34FF34FF34FF34FF34FF34F134F13464
:10002000F134F234F234F334F434F534F634F83491
:1000300010341234163420342534323440345034E1
:1000400064348207F634F834103412341634203411
:100050002534323440345034643480340034253410
:1000600060340034503420340034003440340034E0
:100070000034503400340034003400340034003490
:10008000003482071F341A341A341A342F342A34B5
:100090002A343A344F344A345A346A348F349A34D6
:1000A00011341334163419342234273432343834AA
:1000B0004534543464348207FF342F344F347F3452
:1000C000FF344F348F345F34FF345F346F347F3408
:1000D000FF345F34FF34FF34FF34FF34FF34FF3428
:1000E000FF34FF34FF34FF34FF3482071F341A34E7
:1000F0001A341A341A341A342F342A342A342A344B
:100100003A343A344F344A345F345A346A347A34A5
:100110008F349F341034113413341434163418349B
:1001200020342234253429343234363440344534B2
:100130005134573464348207FF341F343F344F3412
:100140006F348F34FF342F345F348F342F346F3457
:10015000FF345F34FF346F344F341F34FF34FF34C7
:10016000FF34FF34FF34FF34FF34FF34FF34FF34F7
:10017000FF34FF34FF34FF34FF34FF34FF34FF34E7
:10018000FF3482073034313432343334343435344C
:1001900036343734383439342E3473342034203400
:1001A0002034203420348207303431343234333434
:1001B00034343534363437343834393441344234D5
:1001C00043344434453446344734B10CB10C3F30E9
:1001D000B105B1030000B10BEA280800B100F93005
:1001E000A0000000A00BF128B10BEF280800A1002F
:1001F0000A30EE20A10BF82808003230A100FF30B1
:10020000A000A00B0129A10BFF280034AB01AC0119
:10021000AA02031C0E29AB0A2C140829AA070800FD
:10022000A0002A08A00B15290800AA071229AA0174
:10023000AF02031CAE0B1E29AA0A1829AF072F080C
:10024000AB002A08AF00AE0108003A0803178D0082
:1002500083168C130C1483120C080313AA000800D5
:1002600087000030860004308600003086000130B0
:10027000EE20080087000030860004308600003041
:1002800086000530EE20080087000130860005302A
:100290008600013086000130EE2008000330860021
:1002A000F030870008004E210F30EE2030303A2128
:1002B00030303A2130303A2138303A2106303A2174
:1002C00001303A210C303A214E2108003808BA009A
:1002D000BA0DBA0DBA0D3A08F839403E3021023055
:1002E0004421043044210F30442102304421143091
:1002F0004421183044211C3044210030442108009E
:10030000BB003B081E3C031C08003808BA000E3036
:100310003B02031D8D2966210800BA0DBA0DBA0DE6
:100320003A08F839403E30213B08AA000530102138
:100330002A08BB000530B9009D293B0803178D0032
:1003400083168C130C1483120C0803134421BB0A6C
:10035000B90B9D2900304421003044210030442154
:100360000800403084000830A500B8010008802152
:100370008030380730213808BB001F3000020319D5
:10038000C92920300002031CC7290008BB003B0814
:100390004421840AB80AA50BB629483084000830E5
:1003A000A5008030403E302100084421840AA50B7E
:1003B000D429080000307202031DE02986220800BB
:1003C000DE010730A5001F30C1000D30C2008130B2
:1003D0003021013044214830302125087102031CAE
:1003E000F329DE155E1625087202031CF9295E1436
:1003F000DE145E084421A50BED2908000830A50095
:100400004030840020308000840AA50B022A083086
:10041000A5004830840020308000840AA50B0B2AF8
:1004200008000830A500B8018030003E30213808AF
:100430004421B80AA50B172A0800FE21B1210800A3
:100440000830A5004830840020308000840AA50BC5
:10045000242A08002022B121080034080120A0002D
:10046000200E0F39C40020080F39C50034082120A0
:10047000A000200E0F39C60020080F39C700080061
:100480003608BF1C41203F1C7520A000200E0F39EC
:10049000C120C80020080F39C120C9003608BF1C80
:1004A0005B203F1C9B20A000200E0F39C120CA00FA
:1004B00020080F39C120CB00080037083F1C632AF1
:1004C0008A1500208A11BF1C682A8A1548208A11C3
:1004D000A000200E0F39C120CC0020080F39C12008
:1004E000CD0037083F1C772A8A1524208A11BF1CAB
:1004F0007C2A8A157D208A11A000200E0F39C12088
:10050000CE0020080F39C120CF0008000F30C100F5
:10051000C20008002D30C800C9002030CA00CB003E
:1005200008002030CC002D30CD00CE00CF000800D8
:100530002030CA00CB002208A000200E0F39D320A3
:10054000C80020080F39D320C90008007308A20092
:10055000982208002030CC00CD002208A000200EF8
:100560000F39D320CE0020080F39D320CF00080048
:10057000AD01483084003B0884070330A500220801
:10058000AA00643006212C18C72A2D1CCD2A2B085E
:10059000D3208000840AA5032D140A3006212C18CC
:1005A000D32A2D1CD82A2B08D3208000840AA50327
:1005B0002A08D3208000840A20308000840AA50BFA
:1005C000DD2A08002208A000200E0F39D320CA001F
:1005D00020080F39D320CB0008002E08A000200EE1
:1005E0000F39D320C80020080F39D320C9002F08A5
:1005F000A000200E0F39D320CA0020080F39D320C5
:10060000CB0008002030CC00CD00CE0059080F39B7
:10061000D320CF0008003130C8002F30C90045304A
:10062000CC005630CD000F30CE00CF00CB003F1CA9
:100630001C2B3230CA0008003330CA00080000000A
:1006400000000000000000000000000000000000AA
:100650000000000000001F151F192C2B1F1183160E
:100660001E088312A300080000301E0703190800AB
:10067000FF30A300080049309F00831680309F00A0
:1006800083120A30EE201F2341309F0083168130F1
:100690009F0083120A30EE20080051309F0083161D
:1006A00001309F0083120A30EE201F231E08A30092
:1006B00041309F00831681309F0083120A30EE2064
:1006C00008000430A000A60CA70CA613A00B632BF7
:1006D0000800A501A701A601A801B0010800831622
:1006E000FF308500F8308600003087008312B501A6
:1006F000BC01BD01A401A5016A30F500F7009F30DF
:10070000E700E9003B30F600F800FB01FC010C308B
:10071000B4000A30B6001630B70041309F0083168F
:1007200081309F008312A2015321FE21B12171303B
:10073000BA0025212A08E7007230BA0025212A08CC
:10074000F5007330BA0025212A08F6007430BA008B
:1007500025212A08E9007530BA0025212A08F7006A
:100760007630BA0025212A08F8007730BA00252112
:100770002A08EF007830BA0025212A08F0007930E5
:10078000BA0025212A08FA007A30BA0025212A0861
:10079000F3007B30BA0025212A08F4007C30BA002F
:1007A00025212A08B4007D30BA0025212A08FC0042
:1007B0007030BA0025212A08BF00861DD825861A68
:1007C000EA2B6430F720861AEA2B9927BD01B50180
:1007D000BC01F401061AF32BFA30F720061AF32BAA
:1007E0008A15F9238A11CC270A303F1C0F30B60036
:1007F00018303F1C2430EC0022303F1C3330ED0019
:10080000FE212D2240225D22B121402D1F232308ED
:10081000A2009822B121FF30EE20861E392C062C32
:100820003230EE20861D122C3230EE20080032309D
:10083000EE20FA30861EEE2008003230EE20FA302C
:10084000061EEE200800861A232C3230EE20861E6B
:10085000272C080016303F1C2130B7008A15BD1C1C
:10086000A9238A118A22BD1CF724BD1C5D22B12157
:1008700010246923FF30A300BD1C412C861DD02C01
:10088000612C861DCE2D861A522CBD18392C6D0870
:100890003702031CB70A5D228A228622F724B1217F
:1008A0001724392C061A612CBD18392C0030370258
:1008B000031DB7035D228A228622F724B1211D245D
:1008C000392C2308A4001F2324082302031C3C2CDA
:1008D000730203183C2C2408A8001030F9002308E8
:1008E000A7070318A60A1F23F90B6F2CBD18852C28
:1008F000FA241030F9002A08A7070318A60A2B08C3
:10090000A702031CA603F90B7B2C61232708A30075
:10091000BD180134F72513268A15F9218A116B08B1
:10092000DE0710303F1C1830DE02EE01031C6E158E
:100930006E19DE015E08F100A8000A30EE20B50154
:100940003C08A9000130BC001F23FA242A08A30791
:100950002B08A3023125B6006E18B6013608F20046
:100960002908BC00B50A72087102031CBB2C71086F
:10097000B6007208A8008A1566228A11DA218A1543
:1009800053228A116E1D6E10E5244022B121392CAC
:10099000861AC82C392C861AC82C861ECD2C392CC8
:1009A000BD1C392C00346E18B70137086D02031CCA
:1009B000EE146D08EE18B7000F306E1CE02C1330EB
:1009C000EE1CE32C1230C30008006E18B601360886
:1009D0006C02031CEE146C08EE18B6000F306E1C8F
:1009E000F22C1330EE1CF52C1230C30008000F302F
:1009F000C30008002308A400AA01AB0100306F0265
:100A0000031D032D08003B236F08E400E601DF010E
:100A1000700835187A08A100230821020319262D31
:100A200021082302031C1D2D2108A3028A15F92188
:100A30008A115E08AA00AB01262D23082102A3001B
:100A40008A15F9218A115E08AB00AA012408A300C7
:100A50007C1D08002A08A0002B08AA002008AB0073
:100A60000800F72513268A15F9218A116B08DE077D
:100A700036083C183708DE02031C6E145E080800B6
:100A8000B2018A159E238A1140225D22B1211024D1
:100A9000861DCE2D1F23FA242A08A3072B08A302A4
:100AA000EE0131253C18572DB700D3245A2DB6003E
:100AB000E524402240225D22B1211430A5000A30F5
:100AC000EE20861DCE2D861A762D32188A2D061E12
:100AD000952D32143C18712D6C083602031CB60A91
:100AE000482D6D083702031CB70A482D061A892DB8
:100AF000B2188A2D861E952DB2143C18842D003014
:100B00003602031DB603482D00303702031DB7031C
:100B1000482DB201AA01861EAA0A061EAA0AAA1810
:100B2000952DA50B5F2DB201482DBC0ABC18BC0148
:100B30008A159E238A11B121861E9C2D061E9C2D8E
:100B4000482D3C1CB7013C18B6018A15B0238A1108
:100B50002A2210243408A400861DC22D861AB82D1E
:100B60001E303402031CB40A2D22B1211724AC2DEF
:100B7000061AAC2D00303402031DB4032D22B1211E
:100B80001D24AC2D243034020319CE2D3408AA00C4
:100B90007C30BA008A15B2208A11CE2DB50A3508EC
:100BA000023C031CB501B518A52D35182A2C402D83
:100BB0008A15C9238A110B23B1211024861DEF2D1C
:100BC000861EE52D061EE52DDE2D3F1C01303F184B
:100BD0000230BF000B23B1211E30F720DE2D3F086D
:100BE000AA007030BA008A15B2208A1108003518A0
:100BF000052E0A303F1C0F30DF0067083F1C7508C8
:100C0000E4007608E600FB01080069083F1C77084D
:100C1000E4007808E60008303F1C0C30DF00FB01E0
:100C2000FC187B1408003408EB003F1C0800340853
:100C3000AA00033006212B08EB000310EB0D003057
:100C40002A0203190800EB0A2A08AC0075083518B7
:100C50007708AA00323006212A08253C031CAB0A7B
:100C60002B082C1CA307AC1CA3020800D901DA0135
:100C7000DB01DC01DD01DE01DF01E001E101E20178
:100C800008003626B201D901A30120223D1D4022D1
:100C90000223B1213230EE20861E4C2E1024BD18C6
:100CA000582E8619562E3D19DA2E822E1F23602EBD
:100CB0002308003C031C602E2A24A000201CDA2EEE
:100CC0003D1D40220223B1211E30A5000A30EE2036
:100CD00086196D2E3D19DA2E822E861A762E32183E
:100CE0007E2E3D19822EB60A32144F2E061A7D2E04
:100CF00032187E2EB60332144F2EB201A50B662E8B
:100D0000B2014F2E3D1D972E00305902031D8C2E2F
:100D10002308A400A801FB012408B6002308B6029A
:100D20003B2328082302031C7B142308A8006430FB
:100D3000A5000A30EE20A50B9E2EDA2E861D992ED8
:100D4000B03084005908840736088000DB07031898
:100D5000DA0A1030840723088000DD070318DC0A54
:100D60003608D300D500D201D4018A158B228A110E
:100D70005108E2070318E10A5008E1073608D300DA
:100D8000D2012308D500D4018A158B228A1151087B
:100D9000E0070318DF0A5008DF070318DE0AD90A44
:100DA0000223B1213D191724A3015908073C031C54
:100DB000DA2E4F2E5908013C031CED2E013059024A
:100DC000031C08003D1D0800EF016F08AA007730E2
:100DD000BA008A15B2208A1108008A15C9208A1122
:100DE0003D19E6013D1908005908A500B0308400FE
:100DF000A2010008B6008A153B228A111030840730
:100E00005E0800020318062F00085E02A2070F30DA
:100E10008402A50BF92E20228A15D7238A110330CC
:100E2000BB00B822B12110248619142F3B232308BC
:100E3000BD1C232FFA007A08AA007930BA008A155F
:100E4000B2208A110800F0007008AA007830BA00B9
:100E50008A15B2208A1108002A22A622B121102464
:100E6000861D462F861A3C2F09307302031CF30A95
:100E7000A622B1211724302F061A302F0130730219
:100E8000031DF303A622B1211D24302F7308AA00ED
:100E90007A30BA008A15B2208A1108002A22B121BC
:100EA00010248619512F4D232308F4007408AA003A
:100EB0007B30BA008A15B2208A1108002A22B1219B
:100EC0001024861D08001F232308A2000030BB0049
:100ED000B822B1211E30A5000A30EE20861D080080
:100EE000A50B6C2F612F8A156F238A110830A5007E
:100EF000A03084000008A000603084022008800038
:100F000060308407840AA50B7A2F08008A156F23A6
:100F10008A110830A500A03084000008A0005830D5
:100F200084022008800058308407840AA50B8D2F86
:100F300008000130BD008A15B9238A113D088627B3
:100F4000B12117241024861DB82F861AAF2F031045
:100F50003D1FBD0D3D088627B1211724A32F061A7A
:100F6000A32F3D1CBD0C3D088627B1211D24A32FB6
:100F70003D1B08003D087327B121BD1DC12F2C2743
:100F80009B2F3D1EC52F4E279B2FBD1EC92F5E27B1
:100F90009B2F41269B2F08004D2323087402031C1E
:100FA00008008A157F238A11B1216430F720FE21C1
:020FB000080037
:101000008207F334F234F134F134FF34FF34FF3427
:10101000FF34FF341A34FF340A34FF34FF34FF3412
:10102000FF34FF34FF34FF34FF34FF34FF34FF3428
:10103000FF34F134F134F234F334F534F73410344E
:10104000153420343034403482070B342B345B3475
:101050002B348B346B344B343B342B345B341B34A8
:101060007B34F234F334F434F634F8341234153477
:101070002234303445346034903425348034503454
:101080005034003450340034003400340034003420
:101090008207F334F234F234F134F134F134FF34B2
:1010A000FF34FF34FF34FF342A34FF341A341A3447
:1010B000FF34F134F134FF34F234FF34FF34FF34C1
:1010C000FF34FF34FF34FF34FF34FF34FF34FF3488
:1010D000FF34FF34FF34FF34F134F134F134F234AF
:1010E000F234F334F434F534F634F8341034123482
:1010F0001634203425343034403482070B345B34CA
:101100000B345B342B340B348B346B345B344B3407
:101110003B345B342B346B342B341B34A334A63474
:10112000F234A534F334F434F534F634F8341034AE
:101130001234153420342534303440345034603483
:1011400080340034253460340034503400340034AA
:10115000003440340034003450340034003400345F
:10116000003400343A0803178D0003132A080317CC
:101170008C0083160C128C130C158C1355308D00BB
:10118000AA308D008C148C18C3280C118312031301
:1011900008003D1DFB016208D3006108D200590818
:1011A000D500D4018B225008E1005108E2005B0811
:1011B000D300D5005A08D200D4008B225108E20295
:1011C000031CE1035008E1026008D3005F08D2006D
:1011D0005908D500D4018B223E08DE005008DF00FC
:1011E0005108E0005B08D3005A08D2005D08D50022
:1011F0005C08D4008B227B180C295108E0020318EC
:1012000005290130DF02031CDE035008DF02031C46
:10121000DE033E08DE0220296008D10203181429EB
:101220000130D002031CBE035F08D002031CBE03C2
:101230005E08BE023E08DE005008DF005108E000F4
:101240005F080A3C03182B29DF0CE00CDF13E10CCC
:10125000E20CE11320296008D3005F08D2001930A6
:10126000D500D4018B225108D3005008D200620867
:10127000D5006108D400BE22AD225108E400500818
:10128000E3006308003C031CE42B3D1D5729640860
:10129000EF006F08AA007730BA00B2207C117B18EB
:1012A0007C157C08AA007D30BA00B22008005D08D9
:1012B000D3005C08D2001930D500D4018B2251082C
:1012C000E6005008E5006408D3006308D2005B081C
:1012D000D5005A08D4008B226608D3006508D200D6
:1012E0005108E602031878290130E502031C7D2924
:1012F0005008E502031C7D29862953085102E600A7
:10130000031CD00352085002E5007B145908D30097
:10131000D2011930D500D4018B226608D3006508AC
:10132000D2005108D5005008D400BE22AD22510889
:10133000E6005008E5003D1CA52964083F18E700B9
:101340003F1CF5006608F600AC2964083F18E90068
:101350003F1CF7006608F80002303F1C0330D50040
:10136000D4016408D300D2018B225108D300500865
:10137000D20003303F1C0230D500D401BE22AD2282
:101380003D1CD72951083F18F5003F1CE7006708AE
:10139000AA007130BA00B2207508AA007230BA00F3
:1013A000B2207608AA007330BA00B22008005108B3
:1013B0003F18F7003F1CE9006908AA007430BA0022
:1013C000B2207708AA007530BA00B2207808AA00C7
:1013D0007630BA00B220FC107B18FC147808AA0002
:1013E0007630BA00B2207C08AA007D30BA00B22064
:1013F00008006408D300D2015F08D500D4018B2215
:101400005108AF005008AE002308D300D2011930B4
:10141000D500D4018B225108AF070318AE0A50083B
:10142000AE076608D300D2011930D500D4018B2253
:101430007B18272A5108AF020318222A0130AE0276
:10144000031C392A5008AE02031C392A2D2A5108E0
:10145000AF070318AE0A5008AE072F08D3002E08B6
:10146000D2006408D500D401BE22AD225108DE00AE
:101470000800DE0108006408D300D2013608D50058
:10148000D4018B225108D3005008D2001930D50066
:10149000D401BE22AD225108DE0066087B1CDE07A7
:1014A0007B18DE0208002808D300D2010330D500E3
:1014B000D4018B225108D3005008D2003608D50041
:1014C000D401BE22AD225108B60708007108D3002E
:1014D000D2010730D500D4018B225108D300500827
:1014E000D2003608D500D401BE22AD225108F10049
:1014F0007208D300D2010730D500D4018B225108E5
:10150000D3005008D2003608D500D401BE22AD2247
:101510005108F2000800BE01D001D1011030D60000
:101520000310D10DD00DBE0D0310D30DD20D031C31
:10153000A52A5508D107013003110318D007031954
:10154000BE0A5408D0070318BE0AD60B902A5008CA
:1015500051070314571C03100800AE0CAF0CAE1358
:101560002E085202031C0800031DBA2A2F0853023A
:10157000031C0800D10F0800D00A08005508AF006E
:101580005408AE00550403190800D001D101013000
:10159000D600D41BD02A0310D50DD40DD60AC92AE3
:1015A0000310D10DD00D5508D3020318DF2A0130E6
:1015B000D2020318DF2AD20A5508D307E42A5408B6
:1015C000D202031CEA2A51140310D40CD50CD60BFA
:1015D000D02A08005508D3070318D20A5408D207A6
:1015E000E42A83164530A0007830A1007030A200B4
:1015F0006F30A3000F30A400A500A600A70083123F
:10160000080083164630A0006C30A1006130A200B3
:101610007330A3006830A4000F30A500A600A70017
:101620008312080083165430A0006530A10070308A
:10163000A2006C30A3006F30A4007430A5006130AC
:10164000A6000F30A7008312080083164330A000C5
:101650006930A1007430A2006C30A3006930A4008E
:101660007630A5002E30A6000F30A70083120800A8
:1016700083164230A0006130A1007430A2006530B2
:10168000A3007230A4006930A5006530A6000F30B9
:10169000A7008312080083165230A0006530A10015
:1016A0006630A2006530A3007230A4006530A5004A
:1016B0006E30A6006330A7008312080083164B30FB
:1016C000A0006F30A1006E30A2006530A30063302F
:1016D000A4000F30A500A600A70083120800A000F8
:1016E0002018F122A018012320191223A019252364
:1016F000201A3823A01A4B23201B5E2308005330E6
:10170000C0006C30C1006130C2006230C300613083
:10171000C4000F30C500C600C7006230C800613089
:10172000C9007430CA006530CB007230CC0069301B
:10173000CD006530CE002030CF0008000D30C00055
:101740000A303C180B30C1000C30C2000F30C3000F
:1017500008000E30C0000F30C100C200C3000800F6
:101760001030C0001130C1000030C2000F30C30083
:1017700008004B30C0004130C1004C30C20049303D
:10178000C3004230C4005230C5000F30C600C7004D
:1017900008004B30C0007230C1006F30C2006B30A7
:1017A000C3000F30C400C500C600C7000800F630F3
:1017B000C8006430C9003D30CA002030CB00CC00E6
:1017C000CD00CE00CF0008004330C0006830C1001B
:1017D0007930C2006230C3006130C4002130C500DE
:1017E0000F30C600C7008A112022B1218A15F72BBD
:1017F00008005030C0006130C1007230C20061305A
:10180000C3006D30C4006530C5007430C60072304E
:10181000C7003D30CB00FB016130C8006530C90016
:101820003230CA006708A2000430BB007B18BB0A34
:101830008A11B8222D307B18CC00B12123248A15BF
:101840006130C8006530C9003330CA007508A20095
:101850000430BB007B18BB0A8A11B8222D307B18DC
:10186000CC00B12123248A152030C8006230C90081
:101870006530CA007608A2000430BB007B18BB0AA2
:101880008A11B8222D307B18CC00B12123248A156F
:101890006130C8006630C9003230CA006908A20051
:1018A0000430BB007B18BB0A8A11B8222D307B188C
:1018B000CC00B12123248A156130C8006630C900EC
:1018C0003330CA007708A2000430BB007B18BB0A83
:1018D0008A11B8222D307B18CC00B12123248A151F
:1018E000FC187B142030C8006230C9006630CA0082
:1018F0007808A2000430BB007B18BB0A8A11B8220A
:101900002D307B18CC00B12123248A15FB017C19D2
:101910007B142030C8006130C9007430CA006F08E1
:10192000A2000430BB007B18BB0A8A11B8222D30FC
:101930007B18CC00B12123248A15FB016330C80039
:101940006530C9007430CA007008A2000430BB00C2
:101950007B18BB0A8A11B8222D307B18CC00B1212C
:1019600023248A156330C8006630C9007430CA0069
:101970007A08A2000430BB007B18BB0A8A11B82287
:0E1980002D307B18CC00B12123248A150800DD
:02400E00313F40
:10420000060009000900090006000200060002007D
:10421000020007000E000100060008000F000E005B
:104220000100060001000E000200040009000F005A
:1042300001000E0008000E0001000E00060008003C
:104240000E00090006000F00010002000400040037
:104250000600090006000900060006000900070024
:10426000010006000600090009000F000900070010
:10427000020002000200020000000000140014000E
:10428000080015000E001F000E00150000000000C1
:10429000000000000000000000000000000000001E
:1042A00002000200020002000200070008000600EF
:1042B00001000E001F001B0011001B001F001F004B
:0842C0001F0011001F001F0088
:1042E00001004D0034006D00380026009D000000E4
:1042F00000000000050000000C00000000000000AD
:00000001FF
